:020000040000FA
:100000006828000000000000A300030EA400ED30EB
:100010008100051185110512271812282008860075
:1000200005151528210886008515A70A0230270224
:100030000319A701A90B22280630A900AA0B222820
:100040000630AA000B11240E8300A30E230E090014
:1000500082073F3406345B344F3466346D347D346C
:1000600007347F346F34FF30A000A100A200FF30BE
:1000700051203B200800A1015E30A000A100030137
:1000800051203030A000A100030151203930A000E0
:10009000A100030151207930A000A10003015120EB
:1000A0000800A800A6010000A60B5328A80B53289F
:1000B0000800A00C031C5E282030A000A10C031C2B
:1000C00063282030A10085140630512085100800D7
:1000D0008B138B1B68288B01831307309F0003133E
:1000E00083160530810086010130850008308E00BE
:1000F0008312851414305120851085018601A701D3
:10010000ED3081008B168B1733200630A900AA0032
:10011000A428FA30A800051C8928A80B8B280518EC
:100120008F282030A000A100592004305120051C48
:1001300094280430AB0059202B0851200230AB0723
:1001400050302B02031C9B2829082820A0002A08D5
:080150002820A1008510892878
:02400E00380276
:00000001FF
